Table of Contents
实验4:
实验4的:
实验2的:
实验3的日志:
Home Database Mysql Tutorial 非IMU模式下一条update语句产生REDORECORD条数的探究

非IMU模式下一条update语句产生REDORECORD条数的探究

Jun 07, 2016 pm 03:23 PM
update model statement

注意: 每个实验前最好做下日志切换,更详细方法dump redo 文件的方法及本篇DUMP的TRACE文件见下载附件:本篇TRACE等附件下载,或者另一篇博客 :非IMU模式下DML语句产生的REDO日志内容式解读 实验1: BYS@ bys3select * from dept; DEPTNO DNAME LOC ------

注意:每个实验前最好做下日志切换,更详细方法dump redo 文件的方法及本篇DUMP的TRACE文件见下载附件:本篇TRACE等附件下载,或者另一篇博客 :非IMU模式下DML语句产生的REDO日志内容格式解读

实验1:

BYS@ bys3>select * from dept;
DEPTNO DNAME LOC
---------- -------------- -------------
10 database NEW YORK
20 database DALLAS
40 OPERATIONS BOSTON
11 database bj
22 test sh
update dept set dname='oracle' where deptno 4 rows updated.

这个更新语句会产生四条REDO RECORD,因为对四条记录改为oracle
#############################

实验2:

BYS@ bys3>select * from dept;
DEPTNO DNAME LOC
---------- -------------- -------------
10 ACCOUNTING NEW YORK
20 RESEARCH DALLAS
40 OPERATIONS BOSTON
11 database bj
22 test sh
BYS@ bys3>update dept set dname='database' where deptno 3 rows updated.
这个更新语句中,已经有一条是database,这次更新了三条语句,但是只有两条REDO RECORD,
有一个REDO RECORD的CHANGE #1不一样:这个REDO RECORD只有CHANGE #1,CHANGE #2,CHANGE #1中就把这两个值放入UNDO,详见后面日志。
##########################################

实验3:

BYS@ bys3>select * from dept;
DEPTNO DNAME LOC
---------- -------------- -------------
10 oracle NEW YORK
20 oracle DALLAS
40 OPERATIONS BOSTON
11 oracle bj
22 oracle sh
BYS@ bys3>set time on
09:47:59 BYS@ bys3>update dept set dname='oracle' where deptno=10;
1 row updated.
将一行中oracle--UPDATE为oracle,一条REDO RECORD
####################

实验4:

10:08:32 BYS@ bys3>select * from dept;
DEPTNO DNAME LOC
---------- -------------- -------------
10 oracle NEW YORK
20 oracle DALLAS
40 OPERATIONS BOSTON
11 oracle bj
22 oracle sh
10:08:57 BYS@ bys3>update dept set dname='oracle' where deptno 4 rows updated.

更新了四行,这四行原值oracle,更新为oracle,只有一条一条REDO RECORD

##################

附dump 每次操作的redo日志

实验1的:

REDO RECORD - Thread:1 RBA: 0x00013b.00000029.0010 LEN: 0x01e4 VLD: 0x05
SCN: 0x0000.00704cb2 SUBSCN: 1 01/06/2014 22:04:42
(LWN RBA: 0x00013b.00000029.0010 LEN: 0003 NST: 0001 SCN: 0x0000.00704cb1)
CHANGE #1 TYP:0 CLS:33 AFN:3 DBA:0x00c00100 OBJ:4294967295 SCN:0x0000.00704c81 SEQ:1 OP:5.2 ENC:0 RBL:0
ktudh redo: slt: 0x0015 sqn: 0x00000e9f flg: 0x0012 siz: 164 fbi: 0
uba: 0x00c02e0e.0247.2a pxid: 0x0000.000.00000000
CHANGE #2 TYP:0 CLS:34 AFN:3 DBA:0x00c02e0e OBJ:4294967295 SCN:0x0000.00704c80 SEQ:3 OP:5.1 ENC:0 RBL:0
ktudb redo: siz: 164 spc: 3160 flg: 0x0012 seq: 0x0247 rec: 0x2a
xid: 0x0009.015.00000e9f
ktubl redo: slt: 21 rci: 0 opc: 11.1 [objn: 22327 objd: 22327 tsn: 4]
Undo type: Regular undo Begin trans Last buffer split: No
Temp Object: No
Tablespace Undo: No
0x00000000 prev ctl uba: 0x00c02e0e.0247.27
prev ctl max cmt scn: 0x0000.007049b5 prev tx cmt scn: 0x0000.007049e3
txn start scn: 0xffff.ffffffff logon user: 32 prev brb: 12591203 prev bcl: 0 BuExt idx: 0 flg2: 0
KDO undo record:
KTB Redo
op: 0x04 ver: 0x01
compat bit: 4 (post-11) padding: 1
op: L itl: xid: 0x0001.00f.00000e9c uba: 0x00c01cbf.0250.0f
flg: C--- lkc: 0 scn: 0x0000.00702fe2
KDO Op code: URP row dependencies Disabled
xtype: XA flags: 0x00000000 bdba: 0x010000fd hdba: 0x010000fa
itli: 1 ispac: 0 maxfr: 4858
tabn: 0 slot: 2(0x2) flag: 0x2c lock: 0 ckix: 0
ncol: 3 nnew: 1 size: 2
col 1: [ 8] 64 61 74 61 62 61 73 65
CHANGE #3 TYP:2 CLS:1 AFN:4 DBA:0x010000fd OBJ:22327 SCN:0x0000.00703bc4 SEQ:1 OP:11.5 ENC:0 RBL:0
KTB Redo
op: 0x11 ver: 0x01
compat bit: 4 (post-11) padding: 1
op: F xid: 0x0009.015.00000e9f uba: 0x00c02e0e.0247.2a
Block cleanout record, scn: 0x0000.00704cb2 ver: 0x01 opt: 0x02, entries follow...
itli: 2 flg: 2 scn: 0x0000.00703bc4
KDO Op code: URP row dependencies Disabled
xtype: XA flags: 0x00000000 bdba: 0x010000fd hdba: 0x010000fa
itli: 1 ispac: 0 maxfr: 4858
tabn: 0 slot: 2(0x2) flag: 0x2c lock: 1 ckix: 0
ncol: 3 nnew: 1 size: -2
col 1: [ 6] 6f 72 61 63 6c 65
##############################################################
REDO RECORD - Thread:1 RBA: 0x00013b.0000002a.0010 LEN: 0x0108 VLD: 0x01
SCN: 0x0000.00704cb2 SUBSCN: 1 01/06/2014 22:04:42
CHANGE #1 TYP:0 CLS:34 AFN:3 DBA:0x00c02e0e OBJ:4294967295 SCN:0x0000.00704cb2 SEQ:1 OP:5.1 ENC:0 RBL:0
ktudb redo: siz: 96 spc: 2994 flg: 0x0022 seq: 0x0247 rec: 0x2b
xid: 0x0009.015.00000e9f
ktubu redo: slt: 21 rci: 42 opc: 11.1 objn: 22327 objd: 22327 tsn: 4
Undo type: Regular undo Undo type: Last buffer split: No
Tablespace Undo: No
0x00000000
KDO undo record:
KTB Redo
op: 0x02 ver: 0x01
compat bit: 4 (post-11) padding: 1
op: C uba: 0x00c02e0e.0247.2a
KDO Op code: URP row dependencies Disabled
xtype: XA flags: 0x00000000 bdba: 0x010000fd hdba: 0x010000fa
itli: 1 ispac: 0 maxfr: 4858
tabn: 0 slot: 3(0x3) flag: 0x2c lock: 0 ckix: 0
ncol: 3 nnew: 1 size: 2
col 1: [ 8] 64 61 74 61 62 61 73 65
CHANGE #2 TYP:0 CLS:1 AFN:4 DBA:0x010000fd OBJ:22327 SCN:0x0000.00704cb2 SEQ:1 OP:11.5 ENC:0 RBL:0
KTB Redo
op: 0x02 ver: 0x01
compat bit: 4 (post-11) padding: 1
op: C uba: 0x00c02e0e.0247.2b
KDO Op code: URP row dependencies Disabled
xtype: XA flags: 0x00000000 bdba: 0x010000fd hdba: 0x010000fa
itli: 1 ispac: 0 maxfr: 4858
tabn: 0 slot: 3(0x3) flag: 0x2c lock: 1 ckix: 0
ncol: 3 nnew: 1 size: -2
col 1: [ 6] 6f 72 61 63 6c 65
###################################################
REDO RECORD - Thread:1 RBA: 0x00013b.0000002a.0118 LEN: 0x0108 VLD: 0x01
SCN: 0x0000.00704cb2 SUBSCN: 1 01/06/2014 22:04:42
CHANGE #1 TYP:0 CLS:34 AFN:3 DBA:0x00c02e0e OBJ:4294967295 SCN:0x0000.00704cb2 SEQ:2 OP:5.1 ENC:0 RBL:0
ktudb redo: siz: 96 spc: 2896 flg: 0x0022 seq: 0x0247 rec: 0x2c
xid: 0x0009.015.00000e9f
ktubu redo: slt: 21 rci: 43 opc: 11.1 objn: 22327 objd: 22327 tsn: 4
Undo type: Regular undo Undo type: Last buffer split: No
Tablespace Undo: No
0x00000000
KDO undo record:
KTB Redo
op: 0x02 ver: 0x01
compat bit: 4 (post-11) padding: 1
op: C uba: 0x00c02e0e.0247.2b
KDO Op code: URP row dependencies Disabled
xtype: XA flags: 0x00000000 bdba: 0x010000fd hdba: 0x010000fa
itli: 1 ispac: 0 maxfr: 4858
tabn: 0 slot: 5(0x5) flag: 0x2c lock: 0 ckix: 0
ncol: 3 nnew: 1 size: 2
col 1: [ 8] 64 61 74 61 62 61 73 65
CHANGE #2 TYP:0 CLS:1 AFN:4 DBA:0x010000fd OBJ:22327 SCN:0x0000.00704cb2 SEQ:2 OP:11.5 ENC:0 RBL:0
KTB Redo
op: 0x02 ver: 0x01
compat bit: 4 (post-11) padding: 1
op: C uba: 0x00c02e0e.0247.2c
KDO Op code: URP row dependencies Disabled
xtype: XA flags: 0x00000000 bdba: 0x010000fd hdba: 0x010000fa
itli: 1 ispac: 0 maxfr: 4858
tabn: 0 slot: 5(0x5) flag: 0x2c lock: 1 ckix: 0
ncol: 3 nnew: 1 size: -2
col 1: [ 6] 6f 72 61 63 6c 65
###################################################################
REDO RECORD - Thread:1 RBA: 0x00013b.0000002b.0030 LEN: 0x0104 VLD: 0x01
SCN: 0x0000.00704cb2 SUBSCN: 1 01/06/2014 22:04:42
CHANGE #1 TYP:0 CLS:34 AFN:3 DBA:0x00c02e0e OBJ:4294967295 SCN:0x0000.00704cb2 SEQ:3 OP:5.1 ENC:0 RBL:0
ktudb redo: siz: 92 spc: 2798 flg: 0x0022 seq: 0x0247 rec: 0x2d
xid: 0x0009.015.00000e9f
ktubu redo: slt: 21 rci: 44 opc: 11.1 objn: 22327 objd: 22327 tsn: 4
Undo type: Regular undo Undo type: Last buffer split: No
Tablespace Undo: No
0x00000000
KDO undo record:
KTB Redo
op: 0x02 ver: 0x01
compat bit: 4 (post-11) padding: 1
op: C uba: 0x00c02e0e.0247.2c
KDO Op code: URP row dependencies Disabled
xtype: XA flags: 0x00000000 bdba: 0x010000fd hdba: 0x010000fa
itli: 1 ispac: 0 maxfr: 4858
tabn: 0 slot: 6(0x6) flag: 0x2c lock: 0 ckix: 0
ncol: 3 nnew: 1 size: -2
col 1: [ 4] 74 65 73 74
CHANGE #2 TYP:0 CLS:1 AFN:4 DBA:0x010000fd OBJ:22327 SCN:0x0000.00704cb2 SEQ:3 OP:11.5 ENC:0 RBL:0
KTB Redo
op: 0x02 ver: 0x01
compat bit: 4 (post-11) padding: 1
op: C uba: 0x00c02e0e.0247.2d
KDO Op code: URP row dependencies Disabled
xtype: XA flags: 0x00000000 bdba: 0x010000fd hdba: 0x010000fa
itli: 1 ispac: 0 maxfr: 4858
tabn: 0 slot: 6(0x6) flag: 0x2c lock: 1 ckix: 0
ncol: 3 nnew: 1 size: 2
col 1: [ 6] 6f 72 61 63 6c 65
################################################提交的日志条目:
REDO RECORD - Thread:1 RBA: 0x00013b.0000002c.0010 LEN: 0x008c VLD: 0x05
SCN: 0x0000.00704cb4 SUBSCN: 1 01/06/2014 22:04:43
(LWN RBA: 0x00013b.0000002c.0010 LEN: 0001 NST: 0001 SCN: 0x0000.00704cb3)
CHANGE #1 TYP:0 CLS:33 AFN:3 DBA:0x00c00100 OBJ:4294967295 SCN:0x0000.00704cb2 SEQ:1 OP:5.4 ENC:0 RBL:0
ktucm redo: slt: 0x0015 sqn: 0x00000e9f srt: 0 sta: 9 flg: 0x2 ktucf redo: uba: 0x00c02e0e.0247.2d ext: 8 spc: 2704 fbi: 0
END OF REDO DUMP

实验2的:

REDO RECORD - Thread:1 RBA: 0x00013a.00000002.0010 LEN: 0x01c0 VLD: 0x05
SCN: 0x0000.00703bc1 SUBSCN: 1 01/06/2014 21:56:03
(LWN RBA: 0x00013a.00000002.0010 LEN: 0002 NST: 0001 SCN: 0x0000.00703bc0)
CHANGE #1 TYP:0 CLS:23 AFN:3 DBA:0x00c000b0 OBJ:4294967295 SCN:0x0000.00703b80 SEQ:1 OP:5.2 ENC:0 RBL:0
ktudh redo: slt: 0x0004 sqn: 0x00000ec7 flg: 0x0012 siz: 168 fbi: 0
uba: 0x00c01ddb.0283.21 pxid: 0x0000.000.00000000
CHANGE #2 TYP:0 CLS:24 AFN:3 DBA:0x00c01ddb OBJ:4294967295 SCN:0x0000.00703b7f SEQ:9 OP:5.1 ENC:0 RBL:0
ktudb redo: siz: 168 spc: 3658 flg: 0x0012 seq: 0x0283 rec: 0x21
xid: 0x0004.004.00000ec7
ktubl redo: slt: 4 rci: 0 opc: 11.1 [objn: 22327 objd: 22327 tsn: 4]
Undo type: Regular undo Begin trans Last buffer split: No
Temp Object: No
Tablespace Undo: No
0x00000000 prev ctl uba: 0x00c01ddb.0283.01
prev ctl max cmt scn: 0x0000.007034c7 prev tx cmt scn: 0x0000.007034f1
txn start scn: 0xffff.ffffffff logon user: 32 prev brb: 12590550 prev bcl: 0 BuExt idx: 0 flg2: 0
KDO undo record:
KTB Redo
op: 0x04 ver: 0x01
compat bit: 4 (post-11) padding: 1
op: L itl: xid: 0x0003.013.00000eac uba: 0x00c01ac7.0250.06
flg: C--- lkc: 0 scn: 0x0000.00702d7a
KDO Op code: URP row dependencies Disabled
xtype: XA flags: 0x00000000 bdba: 0x010000fd hdba: 0x010000fa
itli: 2 ispac: 0 maxfr: 4858
tabn: 0 slot: 2(0x2) flag: 0x2c lock: 0 ckix: 0
ncol: 3 nnew: 1 size: 2 ---ACCOUNTING 比database多两个字节
col 1: [10] 41 43 43 4f 55 4e 54 49 4e 47 ---对应的是将第一行第二列的值放进UNDO---ACCOUNTING
CHANGE #3 TYP:0 CLS:1 AFN:4 DBA:0x010000fd OBJ:22327 SCN:0x0000.00703bb3 SEQ:3 OP:11.5 ENC:0 RBL:0
KTB Redo
op: 0x01 ver: 0x01
compat bit: 4 (post-11) padding: 1
op: F xid: 0x0004.004.00000ec7 uba: 0x00c01ddb.0283.21
KDO Op code: URP row dependencies Disabled
xtype: XA flags: 0x00000000 bdba: 0x010000fd hdba: 0x010000fa
itli: 2 ispac: 0 maxfr: 4858
tabn: 0 slot: 2(0x2) flag: 0x2c lock: 2 ckix: 0
ncol: 3 nnew: 1 size: -2
col 1: [ 8] 64 61 74 61 62 61 73 65

REDO RECORD - Thread:1 RBA: 0x00013a.00000002.01d0 LEN: 0x0190 VLD: 0x01 --这个REDO RECORD只有CHANGE #1,CHANGE #2
SCN: 0x0000.00703bc1 SUBSCN: 1 01/06/2014 21:56:03
CHANGE #1 TYP:0 CLS:24 AFN:3 DBA:0x00c01ddb OBJ:4294967295 SCN:0x0000.00703bc1 SEQ:1 OP:5.1 ENC:0 RBL:0
ktudb redo: siz: 164 spc: 3488 flg: 0x0022 seq: 0x0283 rec: 0x22
xid: 0x0004.004.00000ec7
ktubu redo: slt: 4 rci: 33 opc: 11.1 objn: 22327 objd: 22327 tsn: 4
Undo type: Regular undo Undo type: Last buffer split: No
Tablespace Undo: No
0x00000000
KDO undo record:
KTB Redo
op: 0x02 ver: 0x01
compat bit: 4 (post-11) padding: 1
op: C uba: 0x00c01ddb.0283.21
Array Update of 2 rows:
tabn: 0 slot: 3(0x3) flag: 0x2c lock: 0 ckix: 0
ncol: 3 nnew: 1 size: 0
KDO Op code: 21 row dependencies Disabled
xtype: XAxtype KDO_KDOM2 flags: 0x00000080 bdba: 0x010000fd hdba: 0x010000fa
itli: 2 ispac: 0 maxfr: 4858
vect = 3
col 1: [ 8] 52 45 53 45 41 52 43 48 ---DUMP('RESEARCH',16)
tabn: 0 slot: 5(0x5) flag: 0x2c lock: 0 ckix: 0
ncol: 3 nnew: 1 size: 0
KDO Op code: 21 row dependencies Disabled
xtype: XAxtype KDO_KDOM2 flags: 0x00000080 bdba: 0x010000fd hdba: 0x010000fa
itli: 2 ispac: 0 maxfr: 4858
vect = 3
col 1: [ 8] 64 61 74 61 62 61 73 65 --DUMP('DATABASE',16)
CHANGE #2 TYP:0 CLS:1 AFN:4 DBA:0x010000fd OBJ:22327 SCN:0x0000.00703bc1 SEQ:1 OP:11.19 ENC:0 RBL:0
KTB Redo
op: 0x02 ver: 0x01
compat bit: 4 (post-11) padding: 1
op: C uba: 0x00c01ddb.0283.22
Array Update of 2 rows:
tabn: 0 slot: 3(0x3) flag: 0x2c lock: 2 ckix: 0
ncol: 3 nnew: 1 size: 0
KDO Op code: 21 row dependencies Disabled
xtype: XAxtype KDO_KDOM2 flags: 0x00000080 bdba: 0x010000fd hdba: 0x010000fa
itli: 2 ispac: 0 maxfr: 4858
vect = 3
col 1: [ 8] 64 61 74 61 62 61 73 65
tabn: 0 slot: 5(0x5) flag: 0x2c lock: 2 ckix: 0
ncol: 3 nnew: 1 size: 0
KDO Op code: 21 row dependencies Disabled
xtype: XAxtype KDO_KDOM2 flags: 0x00000080 bdba: 0x010000fd hdba: 0x010000fa
itli: 2 ispac: 0 maxfr: 4858
vect = 3
col 1: [ 8] 64 61 74 61 62 61 73 65
REDO RECORD - Thread:1 RBA: 0x00013a.00000004.0010 LEN: 0x008c VLD: 0x05 --这个是提交语句的。
SCN: 0x0000.00703bc4 SUBSCN: 1 01/06/2014 21:56:07
(LWN RBA: 0x00013a.00000004.0010 LEN: 0001 NST: 0001 SCN: 0x0000.00703bc3)
CHANGE #1 TYP:0 CLS:23 AFN:3 DBA:0x00c000b0 OBJ:4294967295 SCN:0x0000.00703bc1 SEQ:1 OP:5.4 ENC:0 RBL:0
ktucm redo: slt: 0x0004 sqn: 0x00000ec7 srt: 0 sta: 9 flg: 0x2 ktucf redo: uba: 0x00c01ddb.0283.22 ext: 16 spc: 3322 fbi: 0

实验3的日志:

REDO RECORD - Thread:1 RBA: 0x00013d.00000002.0010 LEN: 0x0214 VLD: 0x05
SCN: 0x0000.0070cae5 SUBSCN: 1 01/07/2014 09:48:10
(LWN RBA: 0x00013d.00000002.0010 LEN: 0002 NST: 0001 SCN: 0x0000.0070cae4)
CHANGE #1 TYP:0 CLS:23 AFN:3 DBA:0x00c000b0 OBJ:4294967295 SCN:0x0000.0070caaa SEQ:1 OP:5.2 ENC:0 RBL:0
ktudh redo: slt: 0x000d sqn: 0x00000ee5 flg: 0x0012 siz: 188 fbi: 0
uba: 0x00c040fa.0286.12 pxid: 0x0000.000.00000000
CHANGE #2 TYP:0 CLS:24 AFN:3 DBA:0x00c040fa OBJ:4294967295 SCN:0x0000.0070caa9 SEQ:3 OP:5.1 ENC:0 RBL:0
ktudb redo: siz: 188 spc: 5884 flg: 0x0012 seq: 0x0286 rec: 0x12
xid: 0x0004.00d.00000ee5
ktubl redo: slt: 13 rci: 0 opc: 11.1 [objn: 22327 objd: 22327 tsn: 4]
Undo type: Regular undo Begin trans Last buffer split: No
Temp Object: No
Tablespace Undo: No
0x00000000 prev ctl uba: 0x00c040fa.0286.0f
prev ctl max cmt scn: 0x0000.0070c50b prev tx cmt scn: 0x0000.0070c522
txn start scn: 0xffff.ffffffff logon user: 32 prev brb: 12599542 prev bcl: 0 BuExt idx: 0 flg2: 0
KDO undo record:
KTB Redo
op: 0x04 ver: 0x01
compat bit: 4 (post-11) padding: 1
op: L itl: xid: 0x0004.004.00000ec7 uba: 0x00c01ddb.0283.22
flg: C--- lkc: 0 scn: 0x0000.00703bc4
Array Update of 1 rows:
tabn: 0 slot: 2(0x2) flag: 0x2c lock: 0 ckix: 0
ncol: 3 nnew: 1 size: 0
KDO Op code: 21 row dependencies Disabled
xtype: XAxtype KDO_KDOM2 flags: 0x00000080 bdba: 0x010000fd hdba: 0x010000fa
itli: 2 ispac: 0 maxfr: 4858
vect = 3
col 1: [ 6] 6f 72 61 63 6c 65
CHANGE #3 TYP:2 CLS:1 AFN:4 DBA:0x010000fd OBJ:22327 SCN:0x0000.00704cb4 SEQ:1 OP:11.19 ENC:0 RBL:0
KTB Redo
op: 0x11 ver: 0x01
compat bit: 4 (post-11) padding: 1
op: F xid: 0x0004.00d.00000ee5 uba: 0x00c040fa.0286.12
Block cleanout record, scn: 0x0000.0070cae5 ver: 0x01 opt: 0x02, entries follow...
itli: 1 flg: 2 scn: 0x0000.00704cb4
Array Update of 1 rows:
tabn: 0 slot: 2(0x2) flag: 0x2c lock: 2 ckix: 0
ncol: 3 nnew: 1 size: 0
KDO Op code: 21 row dependencies Disabled
xtype: XAxtype KDO_KDOM2 flags: 0x00000080 bdba: 0x010000fd hdba: 0x010000fa
itli: 2 ispac: 0 maxfr: 4858
vect = 3
col 1: [ 6] 6f 72 61 63 6c 65

REDO RECORD - Thread:1 RBA: 0x00013d.00000004.0010 LEN: 0x008c VLD: 0x05
SCN: 0x0000.0070cae7 SUBSCN: 1 01/07/2014 09:48:11
(LWN RBA: 0x00013d.00000004.0010 LEN: 0001 NST: 0001 SCN: 0x0000.0070cae6)
CHANGE #1 TYP:0 CLS:23 AFN:3 DBA:0x00c000b0 OBJ:4294967295 SCN:0x0000.0070cae5 SEQ:1 OP:5.4 ENC:0 RBL:0
ktucm redo: slt: 0x000d sqn: 0x00000ee5 srt: 0 sta: 9 flg: 0x2 ktucf redo: uba: 0x00c040fa.0286.12 ext: 19 spc: 5694 fbi: 0

实验4的:

REDO RECORD - Thread:1 RBA: 0x00013f.000000de.0010 LEN: 0x0304 VLD: 0x05
SCN: 0x0000.0070cfe9 SUBSCN: 1 01/07/2014 10:09:20
(LWN RBA: 0x00013f.000000de.0010 LEN: 0002 NST: 0001 SCN: 0x0000.0070cfe8)
CHANGE #1 TYP:0 CLS:33 AFN:3 DBA:0x00c00100 OBJ:4294967295 SCN:0x0000.0070cfbf SEQ:1 OP:5.2 ENC:0 RBL:0
ktudh redo: slt: 0x0004 sqn: 0x00000ebc flg: 0x0012 siz: 308 fbi: 0
uba: 0x00c037d5.0249.08 pxid: 0x0000.000.00000000
CHANGE #2 TYP:0 CLS:34 AFN:3 DBA:0x00c037d5 OBJ:4294967295 SCN:0x0000.0070cfbe SEQ:3 OP:5.1 ENC:0 RBL:0
ktudb redo: siz: 308 spc: 7252 flg: 0x0012 seq: 0x0249 rec: 0x08
xid: 0x0009.004.00000ebc
ktubl redo: slt: 4 rci: 0 opc: 11.1 [objn: 22327 objd: 22327 tsn: 4]
Undo type: Regular undo Begin trans Last buffer split: No
Temp Object: No
Tablespace Undo: No
0x00000000 prev ctl uba: 0x00c037d5.0249.05
prev ctl max cmt scn: 0x0000.0070cc57 prev tx cmt scn: 0x0000.0070cc81
txn start scn: 0xffff.ffffffff logon user: 32 prev brb: 12597202 prev bcl: 0 BuExt idx: 0 flg2: 0
KDO undo record:
KTB Redo
op: 0x04 ver: 0x01
compat bit: 4 (post-11) padding: 1
op: L itl: xid: 0x0004.00d.00000ee5 uba: 0x00c040fa.0286.12
flg: C--- lkc: 0 scn: 0x0000.0070cae7
Array Update of 4 rows:
tabn: 0 slot: 2(0x2) flag: 0x2c lock: 0 ckix: 0
ncol: 3 nnew: 1 size: 0
KDO Op code: 21 row dependencies Disabled
xtype: XAxtype KDO_KDOM2 flags: 0x00000080 bdba: 0x010000fd hdba: 0x010000fa
itli: 2 ispac: 0 maxfr: 4858
vect = 3
col 1: [ 6] 6f 72 61 63 6c 65
tabn: 0 slot: 3(0x3) flag: 0x2c lock: 0 ckix: 0
ncol: 3 nnew: 1 size: 0
KDO Op code: 21 row dependencies Disabled
xtype: XAxtype KDO_KDOM2 flags: 0x00000080 bdba: 0x010000fd hdba: 0x010000fa
itli: 2 ispac: 0 maxfr: 4858
vect = 3
col 1: [ 6] 6f 72 61 63 6c 65
tabn: 0 slot: 5(0x5) flag: 0x2c lock: 0 ckix: 0
ncol: 3 nnew: 1 size: 0
KDO Op code: 21 row dependencies Disabled
xtype: XAxtype KDO_KDOM2 flags: 0x00000080 bdba: 0x010000fd hdba: 0x010000fa
itli: 2 ispac: 0 maxfr: 4858
vect = 3
col 1: [ 6] 6f 72 61 63 6c 65
tabn: 0 slot: 6(0x6) flag: 0x2c lock: 0 ckix: 0
ncol: 3 nnew: 1 size: 0
KDO Op code: 21 row dependencies Disabled
xtype: XAxtype KDO_KDOM2 flags: 0x00000080 bdba: 0x010000fd hdba: 0x010000fa
itli: 2 ispac: 0 maxfr: 4858
vect = 3
col 1: [ 6] 6f 72 61 63 6c 65
CHANGE #3 TYP:2 CLS:1 AFN:4 DBA:0x010000fd OBJ:22327 SCN:0x0000.0070cb7f SEQ:1 OP:11.19 ENC:0 RBL:0
KTB Redo
op: 0x11 ver: 0x01
compat bit: 4 (post-11) padding: 1
op: F xid: 0x0009.004.00000ebc uba: 0x00c037d5.0249.08
Block cleanout record, scn: 0x0000.0070cfe9 ver: 0x01 opt: 0x02, entries follow...
itli: 1 flg: 2 scn: 0x0000.0070cb7f
Array Update of 4 rows:
tabn: 0 slot: 2(0x2) flag: 0x2c lock: 2 ckix: 0
ncol: 3 nnew: 1 size: 0
KDO Op code: 21 row dependencies Disabled
xtype: XAxtype KDO_KDOM2 flags: 0x00000080 bdba: 0x010000fd hdba: 0x010000fa
itli: 2 ispac: 0 maxfr: 4858
vect = 3
col 1: [ 6] 6f 72 61 63 6c 65
tabn: 0 slot: 3(0x3) flag: 0x2c lock: 2 ckix: 0
ncol: 3 nnew: 1 size: 0
KDO Op code: 21 row dependencies Disabled
xtype: XAxtype KDO_KDOM2 flags: 0x00000080 bdba: 0x010000fd hdba: 0x010000fa
itli: 2 ispac: 0 maxfr: 4858
vect = 3
col 1: [ 6] 6f 72 61 63 6c 65
tabn: 0 slot: 5(0x5) flag: 0x2c lock: 2 ckix: 0
ncol: 3 nnew: 1 size: 0
KDO Op code: 21 row dependencies Disabled
xtype: XAxtype KDO_KDOM2 flags: 0x00000080 bdba: 0x010000fd hdba: 0x010000fa
itli: 2 ispac: 0 maxfr: 4858
vect = 3
col 1: [ 6] 6f 72 61 63 6c 65
tabn: 0 slot: 6(0x6) flag: 0x2c lock: 2 ckix: 0
ncol: 3 nnew: 1 size: 0
KDO Op code: 21 row dependencies Disabled
xtype: XAxtype KDO_KDOM2 flags: 0x00000080 bdba: 0x010000fd hdba: 0x010000fa
itli: 2 ispac: 0 maxfr: 4858
vect = 3
col 1: [ 6] 6f 72 61 63 6c 65

REDO RECORD - Thread:1 RBA: 0x00013f.000000df.0124 LEN: 0x0060 VLD: 0x01
SCN: 0x0000.0070cfea SUBSCN: 1 01/07/2014 10:09:20
CHANGE #1 TYP:0 CLS:33 AFN:3 DBA:0x00c00100 OBJ:4294967295 SCN:0x0000.0070cfe9 SEQ:1 OP:5.4 ENC:0 RBL:0
ktucm redo: slt: 0x0004 sqn: 0x00000ebc srt: 0 sta: 9 flg: 0x2 ktucf redo: uba: 0x00c037d5.0249.08 ext: 10 spc: 6942 fbi: 0

Statement of this Website
The content of this article is voluntarily contributed by netizens, and the copyright belongs to the original author. This site does not assume corresponding legal responsibility. If you find any content suspected of plagiarism or infringement, please contact admin@php.cn

Hot AI Tools

Undresser.AI Undress

Undresser.AI Undress

AI-powered app for creating realistic nude photos

AI Clothes Remover

AI Clothes Remover

Online AI tool for removing clothes from photos.

Undress AI Tool

Undress AI Tool

Undress images for free

Clothoff.io

Clothoff.io

AI clothes remover

Video Face Swap

Video Face Swap

Swap faces in any video effortlessly with our completely free AI face swap tool!

Hot Tools

Notepad++7.3.1

Notepad++7.3.1

Easy-to-use and free code editor

SublimeText3 Chinese version

SublimeText3 Chinese version

Chinese version, very easy to use

Zend Studio 13.0.1

Zend Studio 13.0.1

Powerful PHP integrated development environment

Dreamweaver CS6

Dreamweaver CS6

Visual web development tools

SublimeText3 Mac version

SublimeText3 Mac version

God-level code editing software (SublimeText3)

What does WeChat's Do Not Disturb mode do? What does WeChat's Do Not Disturb mode do? Feb 23, 2024 pm 10:48 PM

What does WeChat Do Not Disturb mode mean? Nowadays, with the popularity of smartphones and the rapid development of mobile Internet, social media platforms have become an indispensable part of people's daily lives. WeChat is one of the most popular social media platforms in China, and almost everyone has a WeChat account. We can communicate with friends, family, and colleagues in real time through WeChat, share moments in our lives, and understand each other’s current situation. However, in this era, we are also inevitably faced with the problems of information overload and privacy leakage, especially for those who need to focus or

What is sleep mode used for on iPhone? What is sleep mode used for on iPhone? Nov 04, 2023 am 11:13 AM

iOS devices have long been able to track your sleep patterns and more using the Health app. But isn’t it annoying when you’re disturbed by notifications while you’re sleeping? These notifications may be irrelevant and therefore disrupt your sleep patterns in the process. While Do Not Disturb mode is a great way to avoid distractions while sleeping, it can cause you to miss important calls and messages you receive during the night. Thankfully, this is where sleep mode comes in. Let’s learn more about it and how to use it on iPhone. What role does sleep mode play on the iPhone? Sleep mode is a dedicated focus mode in iOS that is automatically activated based on your sleep schedule in the "Health" App. It helps you set an alarm and then

How to enable/disable VS Code automatic updates How to enable/disable VS Code automatic updates Apr 28, 2023 am 09:28 AM

If you are using Visual Studio Code (VSCode) and thinking about how to disable its automatic software updates and how to disable the automatic updates of its extensions, then read this article. If you don't use VSCode often, open the editor after a long period of time and want to enable automatic updates, this article will also guide you in doing so. Let us discuss in detail the different ways to enable or disable VSCode automatic updates. Table of Contents Method One: Use Settings to Enable/Disable VSCode Automatic Updates Step 1: Open VS Code and click the gear-shaped symbol in the lower left corner. Step 2: Click Settings in the list that appears. Step 3: Type update in the search bar and hit enter. Find Updates: Pattern 4

Do Not Disturb Mode Not Working in iPhone: Fix Do Not Disturb Mode Not Working in iPhone: Fix Apr 24, 2024 pm 04:50 PM

Even answering calls in Do Not Disturb mode can be a very annoying experience. As the name suggests, Do Not Disturb mode turns off all incoming call notifications and alerts from emails, messages, etc. You can follow these solution sets to fix it. Fix 1 – Enable Focus Mode Enable focus mode on your phone. Step 1 – Swipe down from the top to access Control Center. Step 2 – Next, enable “Focus Mode” on your phone. Focus Mode enables Do Not Disturb mode on your phone. It won't cause any incoming call alerts to appear on your phone. Fix 2 – Change Focus Mode Settings If there are some issues in the focus mode settings, you should fix them. Step 1 – Open your iPhone settings window. Step 2 – Next, turn on the Focus mode settings

iPhone 15 Pro: How to get rid of the silent mode symbol in the status bar iPhone 15 Pro: How to get rid of the silent mode symbol in the status bar Sep 24, 2023 pm 10:01 PM

On iPhone 15 Pro and iPhone 15 Pro Max models, Apple introduced a physically programmable action button that replaces the traditional ring/silent switch above the volume buttons. The action button can be programmed to perform several different functions, but the ability to switch between silent and ring modes isn't gone. By default, a long press on the action button will silence the device and the button's tactile feedback will pulse three times. Both iPhone 15 Pro models will display a crossed-out bell symbol next to the time in the status bar to indicate that silent/silent mode is activated, and it will remain so until you long-press the Action button again to unmute the device. If you prefer to put your iPhone in silent mode

KDE Plasma 6.1 brings many enhancements to the popular Linux desktop KDE Plasma 6.1 brings many enhancements to the popular Linux desktop Jun 23, 2024 am 07:54 AM

After several pre-releases, the KDE Plasma development team unveiled version 6.0 of its desktop environment for Linux and BSD systems on 28 February, using the Qt6 framework for the first time. KDE Plasma 6.1 now comes with a number of new features t

How to leave S mode on Windows 10/11 How to leave S mode on Windows 10/11 Aug 03, 2023 pm 08:17 PM

Windows in S mode is designed to provide enhanced security and performance by only allowing the installation of apps from the Microsoft Store. While this feature helps prevent malware and ensure a secure computing environment, it may limit users who want to install applications from sources other than the Microsoft Store. If you find yourself in this situation and keep asking yourself how to switch out of S mode in Windows 10/11, then you have come to the right place as we will walk you through how to switch out in Windows 10/11 using two different methods Steps to S Mode ensure you can enjoy the freedom of installing apps from anywhere you choose. Learn how to switch out of S mode in Windows

How to enable 'Notepad++ Dark Mode' and 'Notepad++ Dark Theme'? How to enable 'Notepad++ Dark Mode' and 'Notepad++ Dark Theme'? Oct 27, 2023 pm 11:17 PM

Notepad++ dark mode v8.0 has no parameters, Notepad++ is the most useful text editor. Every app running on Windows 10 supports dark mode. You can name web browsers such as Chrome, Firefox, and Microsoft Edge. If you work on Notepad++, the default white background may hurt your eyes. Developers have added dark mode to version 8 of Notepad++, here's how to turn it on. Enable Notepad for Windows 11/10 ++ Dark Mode Launch Notepad ++ Click "Settings" > "Preferences" > "Dark Mode" Select "Enable Dark Mode" to restart Notepad

See all articles